:10000000b6c0fecffdcffccffbcffacff9cff8cff4
:10001000f7cff6cf4351204351204445205541317d
:1000200041434f2f422055413141434f2f42204cf5
:100030004f43204b4f343952502023232323232373
:100040002323232323232323232323232323232380
:100050002323232323232323232323232323232370
:100060002323232323232323232323232323232360
:100070002323232323232323232323232323232350
:100080002323232323232323232323232323232340
:100090002300010000010001010101010001010133
:1000a0000100000101010000000101000000000149
:1000b000000000000001000000000101000000013c
:1000c0000101000001010101000202020505020216
:1000d00002050502020205050202020505020202ee
:1000e00005050202020505020202050500010505db
:1000f00005010000000501000100050100000505e3
:1001000000050505050000010005010100050500c9
:1001100000000005000005050500010101050100c2
:1001200001050500010000050101050505010005a7
:10013000050501010105050001010005010100019e
:100140000500010005050000000505010505050580
:100150000000010505000000010500010105050181
:100160000000010501000101050101000005f894ee
:10017000ee27ecbbe5bff8e1a4b7a77fa4bff1bdb4
:10018000e1bd8de0a2e0ed938a95e9f780e4a0e679
:10019000ed938a95e9f7efe9edbfc0e769c0cfd0ed
:1001a00000e0003808f061c02197e02fab81bc81ee
:1001b00090d091d0c895e02de883a881a33211f4a6
:1001c000219653c0a881aa3249f488d0e8eef3e022
:1001d00089d08bd0e0e5f0e085d044c0a881a03282
:1001e00011f4ede3e883a881af3210f0ab3508f0ed
:1001f00039c02497ec81ef526cd0ea83fb83a5e0f1
:10020000b0e08dd0e883f98374d0ac3de0e0be0768
:1002100010f0259628c010e0153000f56dd0c89577
:10022000e02de03031f45ad0e0e5f0e05bd05dd075
:1002300010c062d0c895a02da13031f44fd0e0efae
:10024000f0e050d052d005c057d0c895a02da230b4
:1002500019f4e0e5f0e046d01f5fdecfe0eff0e01c
:1002600041d0249621960f5f9ccf6cd024960895a0
:10027000e0e0e8bbefe3e7bbe2e1efbde3e0e3bfd3
:10028000e0e0e2bfe0e8e6bfe0e0e9bdebbfe5bfec
:10029000e9bfe0e8e8b9e0e0e3b9e2e0efbd2197cb
:1002a000e0e0e883a881a33070f4e4e1f0e0fa93a1
:1002b000ea9375dfc29aecedf5e014d0c298e881bc
:1002c000ef5fe883efcfe0e1f7e20cd02196e7cfd4
:1002d000ffcff0e00895ea0ffb1f0895c09ae2e116
:1002e000efbd0895fa93ea930ec0c098e2e0efbd27
:1002f0000895a881b9810895e12ffbdfeadfebdfe4
:10030000ee56ff4f0895e991f991309639f080e665
:1003100099e00197f1f7a8953197c9f708950a2e4a
:100320001b2e81e1aa27bb1b05c010f4a00db11d37
:10033000b695a795f795e7958a95b9f708951a9315
:0a0340000a930895198108810895b9
:00000001ff
